:10000000370101006520A948730000008280148137
:10001000988133E6E60009C685050505E389E6FE15
:1000200013351600828052B82A84452C2A947524F0
:10003000E36F85FE52BE4EB822F44AF0692435C102
:100040001309400693045006130440079309300631
:1000500019A0952C39C50145612C0808C1450A86AF
:10006000C146BD2403450101E31525FF03451101E8
:10007000E31195FE03452101E31D85FC0345310194
:10008000E31995FC03454101E31535FD0345510195
:10009000E31185FC034561014DFD0545227402799C
:1000A0004EBE0545B124227402794EBC4EB80111F2
:1000B000A2E4CAE052FC5AF862F46AF01305203355
:1000C000F522130460369305C0362285C52A9309AC
:1000D0000037930550374E85D52213059037930589
:1000E000E037E92A0924930B4006130C5006930DC0
:1000F000400713093006930C8040130D4041930ACA
:100100007041130510385D220545DD221305703856
:10011000712A552A21C50145E12A0808C1450A86E8
:10012000C1467D2203450101E31575FF0345110119
:10013000E31185FF03452101E31DB5FD03453101B1
:10014000E31985FD03454101E31525FD03455101F3
:10015000E311B5FD034561014DFD21A00545492A87
:100160004DBF1305803999220145592222859305F7
:10017000903BA9221305003C152A852293042500F3
:10018000A92AE36F95FE4E859305F03C052A1305D9
:10019000203D292A9922930425008122E36F95FEB0
:1001A00022859305C03D192A1305003E0122352200
:1001B000930435001D22E36F95FE130590379305D8
:1001C000C03EED281305103FD520012A93044500B9
:1001D0002922E36F95FE4E8A4E8593055037F92804
:1001E0001305D03FE1200122BD4909A80545092298
:1001F0000145FD28FD1913F5F90F3DC913FBF90F52
:1002000066856D205A8579286A854D20F9209304EA
:100210001500E120E36F95FE7D2069D90145C928CD
:100220000808C1450A86C146652003450101E3155A
:1002300075FF03451101E31185FF03452101E31D0E
:10024000B5FD03453101E31985FD03454101E31582
:1002500025FD03455101E311B5FD034561014DFD48
:100260004128512056859920E14913F5F90F59F598
:100270001305C0422528130590379305E0373D2824
:10028000130570432520912893042500B920E36FBE
:1002900095FE22859305C03615201305104439209C
:1002A000D28985B58548730000008280914873002B
:1002B00000008280AD48730000008280930810081F
:1002C0007300000082809308500873000000828051
:1002D00093087008730000008280732510C082802C
:1002E000732500C08280930860087300000082803C
:1002F0000589F322008093920248B3E2A200739032
:100300000280828095487300000082809308000874
:10031000730000008280A14873000000828093086F
:1003200030087300000082809308400873000000CA
:1003300082805261696C726F61642043726F737363
:10034000696E670A666F72205256436F6E74726FE1
:100350006C6C65720A496E697469616C697A696E60
:10036000672048570A006C69676874004F4646006A
:1003700062656C6C006F666600676174650075701D
:100380000049646C650A004C696768747765696741
:1003900068743A204F6E0A00547261696E20646579
:1003A0007465637465640A4C696768747765696726
:1003B00068743A204F66660A0059454C4C4F570006
:1003C0004C696768743A2059656C6C6F770A006FE6
:1003D0006E0042656C6C3A204F6E0A005245440034
:1003E0004C696768743A205265640A00646F776EDE
:1003F00000476174653A20446F776E0A0042656C6D
:100400006C3A204F66660A0054696D656F757420FA
:10041000696E2000730A0054696D6520726573650A
:100420007420627920747261696E0A0054696D6586
:1004300064206F75740A00476174653A2055700A2C
:0D044000004C696768743A204F66660A0038
:00000001FF
